:1000000010C017C016C015C014C013C012C011C054
:1000100010C00FC00EC00DC00CC00BC00AC009C07C
:1000200008C011241FBECFE5D1E0DEBFCDBF02D096
:1000300025C0E6CFBA9A90E09F5F9B3018F49111EB
:1000400002C01AC092E080E0EFE4F3EC3197F1F7E0
:1000500000C000008F5F8917B8F30BC0EFE4F3EC2A
:100060003197F1F700C000008F5F8917B8F3C29A8B
:10007000E3CFC29880E0F2CFC298F9CFF894FFCFD7
:00000001FF
